:100000009528000000000000182882070E340D34E7
:100010000B340734C03066001030650003306200D6
:10002000A0308B00F4309200063093009A01080053
:100030009500030E9600900A1008033991000C3EBB
:10004000840000088500110805208600920B3028E6
:100050003620F4309200930B302806309300920A39
:10006000160E8300960E160E0B110900141C0800C4
:100070008C030C0F482809308C008D030D0F482885
:1000800005308D008E030E0F482809308E008F0337
:100090008C08031D08008D08031D08008E08031D31
:1000A00008008F08031D0800940119140800890036
:1000B0008316081483120808080001301A07572015
:1000C0008C0002301A0757208D0003301A07572082
:1000D0008E0004301A0757208F000800831688010D
:1000E000081555308900AA308900881488187628A8
:1000F00008150812831208000C08880001301A073E
:1001000089006E200D08880002301A0789006E20D1
:100110000E08880003301A0789006E200F08880037
:1001200004301A0789006E2008000A205D20141090
:100130001910BE20C420CA20861FA328061FD0285D
:10014000051E16299C28BE20F4309200810114144B
:10015000861F96281918AD28A82806128616023080
:1001600027210616861202302721861BAD2826215C
:10017000861BAD2806128612BE209628861FBE2832
:100180002621861FBE280800061FC4282621061F18
:10019000C4280800051ECA282621051ECA280800F2
:1001A000C4200A308F008E008D008C008F01323009
:1001B00097002621061FE428970BD9288F0A0A30BA
:1001C0000F020319D628D728C4208E013230970099
:1001D0002621061FF328970BE8288E0A0A300E0204
:1001E0000319E528E628C4208D0132309700262126
:1001F000061F0229970BF7288D0A06300D020319F6
:10020000F428F528C4208C01323097002621061FDF
:100210001129970B06298C0A0A300C0203190329AD
:1002200004298B137C208B17C4209C2804309A0748
:100230003C301A0203199A01003089001A0888001C
:100240008B136E208B175D20CA209C2820309800CD
:10025000F8302F210000980B28290800F930FF3EC4
:06026000031D2F29080018
:1042000000000100000000000000020000000000AB
:104210000000030000000000000004000000000097
:104220000000050000000000000006000000000083
:10423000000007000000000000000800000000006F
:104240000000090000000000000000000100000064
:104250000000010001000000000002000100000059
:104260000000030001000000000004000100000045
:0A427000000005000100000000003E
:00000001FF
